:100000001DC037C036C035C034C033C032C031C067
:1000100030C02FC02EC02DC02CC02BC02AC029C07C
:1000200028C027C026C025C024C023C022C021C0AC
:1000300020C01FC01EC01DC01CC01BC011241FBE7D
:10004000CFEFD1E0DEBFCDBF11E0A0E0B1E0EEEB3D
:10005000F1E002C005900D92AE30B107D9F721E072
:10006000AEE0B1E001C01D92A431B207E1F756D075
:10007000A4C0C6CF982F8091B0009093B00090910B
:10008000B10097FFFCCF0895F5DF81E090E008957F
:100090008A3010F4805D01C0895CECCFCF93C82F0B
:1000A00082958F70F5DF8C2F8F70CF91F1CFCF932A
:1000B000C82F892FF3DF8C2FCF91F0CF8AB38F7A9F
:1000C0008ABBD59A80E48093B20080E091E090935F
:1000D0001101809310010895CF93DF93843F19F4A9
:1000E0006093740018C0863F31F4CCB5DDB58D2F18
:1000F000C1DF8C2F05C0883F31F4862F90E047D0B8
:10010000DF91CF91B7CF90EE980F903220F490E02E
:10011000DF91CF9144C0DF91CF910895CF93DF93CA
:10012000CDB7DEB728970FB6F894DEBF0FBECDBFB0
:10013000F89488ED8093710010927300BFDF78947B
:100140001FBC83E08EBD10E080E094DF1F5F912F25
:100150009770E1E0F0E0EC0FFD1FE90FF11D8083E7
:100160008F3F91F7E12FF0E0DF011197A770BB27D8
:1001700081E090E08C0F9D1FA80FB91F3297E770A8
:10018000FF27E80FF91F6C918081A6DFDDCFE19991
:10019000FECF1FBA8EBBE09A99278DB30895262F04
:1001A000E199FECF1CBA1FBA8EBB2DBB0FB6F894D7
:0E01B000E29AE19A0FBE01960895F894FFCFEF
:0E01BE000000000200000000440000000000ED
:00000001FF
